:100000008A110A120528000009000730990083169A
:100010000510851005118312F430A0000130A100F5
:100020000A212F20AC012C08053C031C2B28AD0114
:100030002D083B3C031C2528E830A0000330A1001C
:100040000A210130AD07031C18281F308305013039
:10005000AC07031C13281F3083050C282E28051419
:10006000F430A0000130A1000A217D20B2207D20C3
:10007000B2207D20C020A120A1207220B2206420C7
:10008000B2209520B2209B20B2208420B22086206E
:10009000C0208920B2207920C0208920B22095205C
:1000A000B2209520B2207620C0206920C020F82000
:1000B0009030A0000130A1000A2105102C30A000D2
:1000C0000130A1000A210800D620D620E720D62042
:1000D0000800E720D620E7200800D620E720D62019
:1000E000D6200800E720E720D6200800E720E720F8
:1000F0000800D620E720E7200800D620D620D6200A
:10010000E7200800D6200800E7200800D620D620E7
:100110000800D620E720E720E720E7200800E720B6
:10012000E720E720E720D6200800E720E720E720A7
:10013000E720E7200800D620D620D620D620D620DB
:1001400008006D20B2207920B2208920B2208220C0
:10015000B2208420C020080005114630A000A10173
:100160000A21080005114630A000A1010A214630ED
:10017000A000A1010A214630A000A1010A21080027
:1001800005114630A000A1010A214630A000A101BE
:100190000A214630A000A1010A214630A000A10199
:1001A0000A214630A000A1010A21080005150530EA
:1001B00084000230AA004B30A0000230A1003C3085
:1001C000A2000030A30045210511AC200800051550
:1001D000053084000230AA004B30A0000230A1009C
:1001E000EE30A2000030A30045210511AC2008002C
:1001F0000515053084000230AA004B30A000023003
:10020000A100FC30A2000430A30045210511AC2060
:1002100008000929A008031915291C21A0030000C2
:1002200000000000000000000A29A10803190800CE
:100230001C21A103A0030A290C30A500A50B1E292F
:10024000000000001230A200A20B2B292D212D212D
:100250000000000008002D2124290D30A400A40B6B
:100260002F29000008001030A8020001031C013EE5
:10027000A902031C08003C290A30A8020001031C43
:10028000013EA902031C08003C292A08800420081A
:10029000A8002108A90033210130A202031CA303F6
:1002A0002A0980052008A8002108A9003321A208F6
:0C02B000031D4529A308031D4529080073
:02400E00C431BB
:00000001FF
